:0200000480007A
:100000006F00C004732F2034930F8000630AFF0336
:10001000930F90006306FF03930FB0006302FF038A
:10002000170F0080130F0FFE63040F0067000F000F
:10003000732F203463540F006F004000136E9E53E3
:10004000171F00002320CFFD6FF09FFF732540F1A5
:100050006310050073251030635805000F00F00F82
:10006000130E100073000000130E00009702000032
:10007000938282F973905230735020307350303035
:1000800073504030970200809382C2F7638C020065
:10009000739052109302B01A739022307323203061
:1000A000E39E62F873500030970200009382420191
:1000B00073901234732540F173002030B710FF00A5
:1000C000938000F093C1F0F0B7FE00FF938EFE0026
:1000D000130E20006396D11DB710F00F938000FF20
:1000E00093C1000FB71EF00F938E0EF0130E300069
:1000F0006398D11BB710FF009380F08F93C1F0700D
:10010000B71EFF00938E0EFF130E4000639AD119A5
:10011000B7F00FF09380F00093C1000FB7FE0FF01F
:10012000938EFE0F130E5000639CD117B7F000FFA3
:100130009380007093C0F070B7FE00FF938EFE00B6
:10014000130E6000639ED01513020000B710F00F6D
:10015000938000FF93C1000F13830100130212006C
:1001600093022000E31452FEB71EF00F938E0EF0A0
:10017000130E70006316D31313020000B710FF00B4
:100180009380F08F93C1F07013000000138301007F
:100190001302120093022000E31252FEB71EFF006A
:1001A000938E0EFF130E8000631CD30F130200000A
:1001B000B7F00FF09380F00093C1000F1300000020
:1001C00013000000138301001302120093022000A9
:1001D000E31052FEB7FE0FF0938EFE0F130E900049
:1001E0006310D30D13020000B710F00F938000FFCF
:1001F00093C1000F1302120093022000E31652FE77
:10020000B71EF00F938E0EF0130EA000639AD10963
:1002100013020000B710FF009380F0FF13000000EE
:1002200093C1F0001302120093022000E31452FE67
:10023000B71EFF00938E0EFF130EB0006392D1071E
:1002400013020000B7F00FF09380F00013000000DD
:100250001300000093C1000F13021200930220004C
:10026000E31252FEB7FE0FF0938EFE0F130EC00086
:100270006398D1039340000F930E000F130ED0002C
:100280006390D003B700FF009380F00F13C0F070AD
:10029000930E0000130EE0006314D001631CC00134
:1002A0000F00F00F63000E00131E1E00136E1E00E1
:1002B000730000000F00F00F130E10007300000019
:0402C000731000C0F7
:1010000000000000000000000000000000000000E0
:1010100000000000000000000000000000000000D0
:1010200000000000000000000000000000000000C0
:1010300000000000000000000000000000000000B0
:081040000000000000000000A8
:040000058000200057
:00000001FF
